:100000000C945B000C9483000C9483000C9483008C
:100010000C9483000C9483000C9483000C94830054
:100020000C9483000C9483000C9483000C94830044
:100030000C9483000C9483000C9483000C94830034
:100040000C947C020C9483000C94FD040C948300AB
:100050000C9483000C9483000C9483000C94830014
:100060000C9483000C948300000024272A000025B0
:10007000282B000023262904040404040404040299
:100080000202020202030303030303010204081035
:100090002040800102040810200102040810200002
:1000A0000000070002010000030406000000000039
:1000B00000000000D40011241FBECFEFD4E0DEBF4B
:1000C000CDBF11E0A0E0B1E0ECE4FBE002C00590A0
:1000D0000D92AA30B107D9F711E0AAE0B1E001C052
:1000E0001D92A03AB107E1F710E0C6EBD0E004C0E2
:1000F0002297FE010E94A005C43BD107C9F70E94C8
:10010000CD000C94A4050C94000080910A010E947B
:100110005C0364E070E00E943A059B0170930D015E
:1001200060930C0140910E0150910F01609100010C
:1001300070910101CB01840F951F281739072CF40A
:10014000461B570B421753079CF0B90182E191E01F
:100150000E944C0280910C0190910D0190930F012F
:1001600080930E016AE070E080E090E00E94E70278
:10017000089540E052EC61E070E082E191E00E947D
:10018000E80064E670E080E090E00E94E70260E052
:1001900080910A010E94CE0308950E941F030E94CD
:1001A000B9000E948500FDCF86E091E09093130195
:1001B000809312010895862F0E94BC0408950E9426
:1001C000F40408950E94D50408950E94C40408957B
:1001D000CB01BA010E9483040895DC01ED91FC91EA
:1001E0000190F081E02D09950895DC01ED91FC91DD
:1001F0000190F081E02D099508950F931F93CF93FF
:10020000DF938C01EB0109C02196D801ED91FC919F
:100210000190F081E02DC801099568816623A1F75E
:10022000DF91CF911F910F9108950F931F938C0130
:10023000DC01ED91FC910190F081E02D6DE00995DC
:10024000D801ED91FC910190F081E02D6AE0C801A8
:1002500009951F910F9108950F931F938C01DC0155
:10026000ED91FC910190F081E02D0995C8010E946B
:1002700015011F910F9108950F931F938C010E94F8
:10028000FD00C8010E9415011F910F9108950F9361
:100290001F938C01DC01ED91FC910190F081E02D28
:1002A0000995C8010E9415011F910F9108952F9281
:1002B0003F924F925F926F927F928F929F92AF92F6
:1002C000BF92CF92DF92EF92FF920F931F93DF9333
:1002D000CF93CDB7DEB7A0970FB6F894DEBF0FBEB1
:1002E000CDBF1C016A017B014115510561057105F6
:1002F00049F4DC01ED91FC910190F081E02D60E387
:10030000099554C0882499245401422E552466240A
:10031000772401E010E00C0F1D1F080D191DC70107
:10032000B601A30192010E944D05F8016083089473
:10033000811C911CA11CB11CC701B601A301920133
:100340000E944D05C901DA016C017D01C114D1047F
:10035000E104F104F1F681E0E82EF12CEC0EFD1E33
:10036000E80CF91C3E010894611C711CD501C40104
:100370000197A109B1096C01C818D90814C0F60188
:10038000EE0DFF1D60816A3010F4605D01C0695C94
:10039000D101ED91FC910190F081E02DC101099511
:1003A0000894E108F1086E147F0449F7A0960FB68F
:1003B000F894DEBF0FBECDBFCF91DF911F910F919B
:1003C000FF90EF90DF90CF90BF90AF909F908F9075
:1003D0007F906F905F904F903F902F9008952AE00C
:1003E0000E94570108950F931F938C010E94EF0103
:1003F000C8010E9415011F910F910895AB0160E0A3
:1004000070E00E94EF0108950F931F938C01AB01E0
:1004100060E070E00E94EF01C8010E9415011F9189
:100420000F910895EF92FF920F931F93CF93DF9355
:10043000EC017A018B0177FF0FC0E881F98101900F
:10044000F081E02D6DE2099510950095F094E0940F
:10045000E11CF11C011D111D2AE0B801A701CE010C
:100460000E945701DF91CF911F910F91FF90EF9064
:1004700008950F931F938C010E941202C8010E94DD
:1004800015011F910F910895AB01662757FD6095E7
:10049000762F0E94120208950F931F938C01AB01D7
:1004A000662757FD6095762F0E941202C8010E94B0
:1004B00015011F910F910895DC012115310541F4BB
:1004C000ED91FC910190F081E02D642F0995089544
:1004D0002A30310519F40E94120208950E94570132
:1004E00008950F931F938C010E945C02C8010E9423
:1004F00015011F910F9108951F920F920FB60F9241
:1005000011242F938F939F93AF93BF9380911401E6
:1005100090911501A0911601B09117018050904C57
:10052000AF4FBF4F8093140190931501A093160114
:10053000B093170127C08091140190911501A091EB
:100540001601B091170180589E43A040B04080939F
:10055000140190931501A0931601B0931701809197
:10056000180190911901A0911A01B0911B010196F7
:10057000A11DB11D8093180190931901A0931A0138
:10058000B0931B018091140190911501A091160167
:10059000B091170181589E43A040B04060F6BF91D2
:1005A000AF919F918F912F910F900FBE0F901F9041
:1005B00018958FB7F8942091180130911901409146
:1005C0001A0150911B018FBFB901CA010895EF9222
:1005D000FF920F931F937B018C018FB7F89440918A
:1005E00018015091190160911A0170911B018FBF80
:1005F0002FB7F8948091180190911901A0911A01D8
:10060000B0911B012FBF841B950BA60BB70B8E154A
:100610009F05A007B10760F31F910F91FF90EF9026
:100620000895019759F0FC01EE0FFF1FEE0FFF1F19
:1006300032978FB7F8943197F1F78FBF0895789478
:1006400084B5826084BD84B5816084BD85B58260D7
:1006500085BD85B5816085BDEEE6F0E08081816075
:100660008083E1E8F0E08081826080838081816026
:100670008083E0E8F0E0808181608083E1EBF0E05E
:10068000808184608083E0EBF0E080818160808302
:10069000EAE7F0E0808184608083808182608083EB
:1006A0008081816080838081806880831092C10016
:1006B00008958093080108958F7090910801929594
:1006C000990F990F907C982B90937C0080917A00E1
:1006D000806480937A0080917A0086FDFCCF20911F
:1006E000780040917900942F80E030E0282B392B5E
:1006F000C90108951F93CF93DF93182FEB0161E099
:100700000E94CE03E12FF0E0E156FF4F8491833049
:1007100051F480918000806880938000D09389009C
:10072000C093880037C0843051F48091800080628B
:1007300080938000D0938B00C0938A002BC08130BF
:1007400029F484B5806884BDC7BD24C0823029F4F3
:1007500084B5806284BDC8BD1DC0863041F48091DF
:10076000B00080688093B000C093B30013C087309E
:1007700041F48091B00080628093B000C093B400D7
:1007800009C0C038D10514F460E001C061E0812FD8
:100790000E94EC03DF91CF911F910895282F30E044
:1007A000C90185579F4FFC01949129583F4FF9018A
:1007B0008491882381F0E82FF0E0E859FF4FE4911D
:1007C000F0E0662329F48081909589238083089541
:1007D0008081892B80830895482F50E0CA0181567B
:1007E0009F4FFC012491CA0185579F4FFC019491B2
:1007F00049585F4FFA0134913323C1F1222331F17B
:10080000233021F4809180008F7705C0243031F4AB
:10081000809180008F7D8093800018C0213019F472
:1008200084B58F7704C0223021F484B58F7D84BDD8
:100830000DC0263021F48091B0008F7705C027309D
:1008400029F48091B0008F7D8093B000E32FF0E019
:10085000E359FF4FE491F0E0662329F480819095FD
:100860008923808308958081892B80830895482F70
:1008700050E0CA0181569F4FFC012491CA0185575F
:100880009F4FFC01949149585F4FFA0134913323F3
:1008900019F420E030E035C0222331F1233021F477
:1008A000809180008F7705C0243031F480918000E2
:1008B0008F7D8093800018C0213019F484B58F7724
:1008C00004C0223021F484B58F7D84BD0DC0263054
:1008D00021F48091B0008F7705C0273029F48091F2
:1008E000B0008F7D8093B000E32FF0E0EE58FF4F13
:1008F000E491F0E0808120E030E0892311F021E0F4
:1009000030E0C9010895EF92FF920F931F937B018E
:100910008C0122E030E040E050E00E946F05205C56
:100920003D4B404F5F4FCA01B901A80197010E949A
:100930006F05C901DA010197A109B109292F3A2FE1
:100940004B2F552747FD5A950196A11DB11D2093A8
:10095000C50081508093C400E1ECF0E080818061AB
:1009600080838081886080838081806880831F91FC
:100970000F91FF90EF900895982F8091C00085FF10
:10098000FCCF9093C600089580911C0190911D01A9
:1009900080589F4F20911E0130911F01821B930BA5
:1009A00060E870E00E943A05089540911E01509160
:1009B0001F0180911C0190911D018417950719F466
:1009C0002FEF3FEF0FC0FA01E05EFE4F2081CA011A
:1009D000019660E870E00E943A0590931F018093B1
:1009E0001E0130E0C901089580911E0190911F0100
:1009F00090931D0180931C0108951F920F920FB6D2
:100A00000F9211242F933F934F935F936F937F9394
:100A10008F939F93AF93BF93EF93FF934091C60043
:100A2000E0911C01F0911D01CF01019660E870E09A
:100A30000E943A059C0180911E0190911F01281788
:100A4000390739F0E05EFE4F408330931D0120935B
:100A50001C01FF91EF91BF91AF919F918F917F9179
:100A60006F915F914F913F912F910F900FBE0F901B
:100A70001F90189597FB092E07260AD077FD04D002
:100A800049D006D000201AF4709561957F4F0895E3
:100A9000F6F7909581959F4F0895A1E21A2EAA1B13
:100AA000BB1BFD010DC0AA1FBB1FEE1FFF1FA2171E
:100AB000B307E407F50720F0A21BB30BE40BF50B1B
:100AC000661F771F881F991F1A9469F760957095A4
:100AD000809590959B01AC01BD01CF01089597FBD6
:100AE000092E05260ED057FD04D0D7DF0AD0001CF2
:100AF00038F450954095309521953F4F4F4F5F4FBB
:100B00000895F6F790958095709561957F4F8F4F7A
:100B10009F4F0895AA1BBB1B51E107C0AA1FBB1F13
:100B2000A617B70710F0A61BB70B881F991F5A9579
:100B3000A9F780959095BC01CD010895EE0FFF1F98
:0C0B40000590F491E02D0994F894FFCF8B
:0A0B4C000A0000000000DB000100B9
:00000001FF
